:0600000002003302179A12
:03000B0002179B3E
:030013000217C60B
:03001B000217C702
:030023000217C8F9
:03002B000217C9F0
:10003300759840758780758921758DFF758BFF7560
:100043008850D299758160758CFA758A0075A8827B
:100053007530007531007580FF75900075A00075CF
:10006300B03F782076FF08B830FA75F0FF7590003E
:10007300C2B77880E670257580FE75A00120A00FB9
:10008300300019C200760890190D1217CA800D208E
:10009300000AD20076089019101217CA7881E67008
:1000A300257580FE75A00220A10F300119C20176CB
:1000B300089019131217CA800D20010AD20176087D
:1000C3009019161217CA7882E670257580FE75A0FE
:1000D3000420A20F300219C20276089019191217D0
:1000E300CA800D20020AD202760890191C1217CA80
:1000F3007883E670257580FE75A00820A30F300372
:1001030019C203760890191F1217CA800D20030A1B
:10011300D20376089019221217CA7884E6702575DF
:1001230080FE75A01020A40F300419C20476089035
:1001330019251217CA800D20040AD20476089019D3
:10014300281217CA7885E670257580FE75A02020D1
:10015300A50F300519C205760890192B1217CA800E
:100163000D20050AD205760890192E1217CA788633
:10017300E670257580FE75A04020A60F300619C2D3
:100183000676089019311217CA800D20060AD20686
:1001930076089019341217CA7887E670257580FEA1
:1001A30075A08020A70F300719C20776089019376A
:1001B3001217CA800D20070AD207760890193A123F
:1001C30017CA7888E670257580FD75A00120A00FF9
:1001D300300819C208760890193D1217CA800D20FD
:1001E300080AD20876089019401217CA7889E6706F
:1001F300257580FD75A00220A10F300919C209766B
:10020300089019431217CA800D20090AD2097608EB
:100213009019461217CA788AE670257580FD75A075
:100223000420A20F300A19C20A760890194912173E
:10023300CA800D200A0AD20A760890194C1217CAEE
:10024300788BE670257580FD75A00820A30F300B11
:1002530019C20B760890194F1217CA800D200B0A8A
:10026300D20B76089019521217CA788CE67025754E
:1002730080FD75A01020A40F300C19C20C760890D5
:1002830019551217CA800D200C0AD20C7608901942
:10029300581217CA788DE670257580FD75A0202049
:1002A300A50F300D19C20D760890195B1217CA807D
:1002B3000D200D0AD20D760890195E1217CA788E9A
:1002C300E670257580FD75A04020A60F300E19C27B
:1002D3000E76089019611217CA800D200E0AD20EED
:1002E30076089019641217CA788FE670257580FD19
:1002F30075A08020A70F300F19C20F7608901967D9
:100303001217CA800D200F0AD20F760890196A12AD
:1003130017CA7890E670257580FB75A00120A00FA1
:10032300301019C210760890196D1217CA800D206B
:10033300100AD21076089019701217CA7891E670D5
:10034300257580FB75A00220A10F301119C211760B
:10035300089019731217CA800D20110AD21176085A
:100363009019761217CA7892E670257580FB75A0EE
:100373000420A20F301219C21276089019791217AD
:10038300CA800D20120AD212760890197C1217CA5D
:100393007893E670257580FB75A00820A30F3013B2
:1003A30019C213760890197F1217CA800D20130AF9
:1003B300D21376089019821217CA7894E6702575BD
:1003C30080FB75A01020A40F301419C21476089076
:1003D30019851217CA800D20140AD21476089019B1
:1003E300881217CA7895E670257580FB75A02020C2
:1003F300A50F301519C215760890198B1217CA80EC
:100403000D20150AD215760890198E1217CA789600
:10041300E670257580FB75A04020A60F301619C223
:100423001676089019911217CA800D20160AD21653
:1004330076089019941217CA7897E670257580FB91
:1004430075A08020A70F301719C217760890199747
:100453001217CA800D20170AD217760890199A121C
:1004630017CA7898E670257580F775A00120A00F4C
:10047300301819C218760890199D1217CA800D20DA
:10048300180AD21876089019A01217CA7899E6703C
:10049300257580F775A00220A10F301919C21976AE
:1004A300089019A31217CA800D20190AD2197608C9
:1004B3009019A61217CA789AE670257580F775A069
:1004C3000420A20F301A19C21A76089019A912171C
:1004D300CA800D201A0AD21A76089019AC1217CACC
:1004E300789BE670257580F775A00820A30F301B55
:1004F30019C21B76089019AF1217CA800D201B0A68
:10050300D21B76089019B21217CA789CE67025752B
:1005130080F775A01020A40F301C19C21C76089018
:1005230019B51217CA800D201C0AD21C760890191F
:10053300B81217CA789DE670257580F775A020203C
:10054300A50F301D19C21D76089019BB1217CA805A
:100553000D201D0AD21D76089019BE1217CA789E67
:10056300E670257580F775A04020A60F301E19C2CE
:100573001E76089019C11217CA800D201E0AD21EBA
:1005830076089019C41217CA789FE670257580F70C
:1005930075A08020A70F301F19C21F76089019C7B6
:1005A3001217CA800D201F0AD21F76089019CA128B
:1005B30017CA78A0E670257580EF75A00120A00FFB
:1005C300302019C22076089019CD1217CA800D2049
:1005D300200AD22076089019D01217CA78A1E670A3
:1005E300257580EF75A00220A10F302119C2217655
:1005F300089019D31217CA800D20210AD221760838
:100603009019D61217CA78A2E670257580EF75A0E7
:100613000420A20F302219C22276089019D912178A
:10062300CA800D20220AD22276089019DC1217CA3A
:1006330078A3E670257580EF75A00820A30F3023FB
:1006430019C22376089019DF1217CA800D20230AD6
:10065300D22376089019E21217CA78A4E67025759A
:1006630080EF75A01020A40F302419C224760890BF
:1006730019E51217CA800D20240AD224760890198E
:10068300E81217CA78A5E670257580EF75A02020BB
:10069300A50F302519C22576089019EB1217CA80C9
:1006A3000D20250AD22576089019EE1217CA78A6CE
:1006B300E670257580EF75A04020A60F302619C27D
:1006C3002676089019F11217CA800D20260AD22621
:1006D30076089019F41217CA78A7E670257580EF8B
:1006E30075A08020A70F302719C22776089019F725
:1006F3001217CA800D20270AD22776089019FA12FA
:1007030017CA78A8E670257580DF75A00120A00FB1
:10071300302819C22876089019FD1217CA800D20B7
:10072300280AD2287608901A001217CA78A9E67008
:10073300257580DF75A00220A10F302919C2297603
:1007430008901A031217CA800D20290AD2297608A5
:10075300901A061217CA78AAE670257580DF75A06D
:100763000420A20F302A19C22A7608901A091217F8
:10077300CA800D202A0AD22A7608901A0C1217CAA8
:1007830078ABE670257580DF75A00820A30F302BAA
:1007930019C22B7608901A0F1217CA800D202B0A44
:1007A300D22B7608901A121217CA78ACE670257508
:1007B30080DF75A01020A40F302C19C22C7608906E
:1007C3001A151217CA800D202C0AD22C7608901AFB
:1007D300181217CA78ADE670257580DF75A0202042
:1007E300A50F302D19C22D7608901A1B1217CA8037
:1007F3000D202D0AD22D7608901A1E1217CA78AE34
:10080300E670257580DF75A04020A60F302E19C233
:100813002E7608901A211217CA800D202E0AD22E86
:100823007608901A241217CA78AFE670257580DF10
:1008330075A08020A70F302F19C22F7608901A2792
:100843001217CA800D202F0AD22F7608901A2A1267
:1008530017CA78B0E670257580BF75A00120A00F78
:10086300303019C2307608901A2D1217CA800D2025
:10087300300AD2307608901A301217CA78B1E6706F
:10088300257580BF75A00220A10F303119C23176C2
:1008930008901A331217CA800D20310AD231760814
:1008A300901A361217CA78B2E670257580BF75A004
:1008B3000420A20F303219C2327608901A39121767
:1008C300CA800D20320AD2327608901A3C1217CA17
:1008D30078B3E670257580BF75A00820A30F303369
:1008E30019C2337608901A3F1217CA800D20330AB3
:1008F300D2337608901A421217CA78B4E670257577
:1009030080BF75A01020A40F303419C2347608902C
:100913001A451217CA800D20340AD2347608901A69
:10092300481217CA78B5E670257580BF75A02020D8
:10093300A50F303519C2357608901A4B1217CA80A5
:100943000D20350AD2357608901A4E1217CA78B69A
:10095300E670257580BF75A04020A60F303619C2FA
:10096300367608901A511217CA800D20360AD236ED
:100973007608901A541217CA78B7E670257580BFA7
:1009830075A08020A70F303719C2377608901A5701
:100993001217CA800D20370AD2377608901A5A12D6
:1009A30017CA78B8E6702575807F75A00120A00F5F
:1009B300303819C2387608901A5D1217CA800D2094
:1009C300380AD2387608901A601217CA78B9E670D6
:1009D3002575807F75A00220A10F303919C23976A1
:1009E30008901A631217CA800D20390AD239760883
:1009F300901A661217CA78BAE6702575807F75A0BB
:100A03000420A20F303A19C23A7608901A691217D5
:100A1300CA800D203A0AD23A7608901A6C1217CA85
:100A230078BBE6702575807F75A00820A30F303B47
:100A330019C23B7608901A6F1217CA800D203B0A21
:100A4300D23B7608901A721217CA78BCE6702575E5
:100A5300807F75A01020A40F303C19C23C7608900B
:100A63001A751217CA800D203C0AD23C7608901AD8
:100A7300781217CA78BDE6702575807F75A020208F
:100A8300A50F303D19C23D7608901A7B1217CA8014
:100A93000D203D0AD23D7608901A7E1217CA78BE01
:100AA300E6702575807F75A04020A60F303E19C2E1
:100AB3003E7608901A811217CA800D203E0AD23E54
:100AC3007608901A841217CA78BFE6702575807F5E
:100AD30075A08020A70F303F19C23F7608901A8770
:100AE3001217CA800D203F0AD23F7608901A8A1245
:100AF30017CA75A000C2B778C0E670257580FE7569
:100B0300900120900F304019C2407608901A8D1240
:100B130017CA800D20400AD2407608901A90121707
:100B2300CA78C1E670257580FE75900220910F305A
:100B33004119C2417608901A931217CA800D2041B9
:100B43000AD2417608901A961217CA78C2E670251F
:100B53007580FE75900420920F304219C2427608C8
:100B6300901A991217CA800D20420AD24276089031
:100B73001A9C1217CA78C3E670257580FE75900813
:100B830020930F304319C2437608901A9F1217CA55
:100B9300800D20430AD2437608901AA21217CA780E
:100BA300C4E670257580FE75901020940F304419AB
:100BB300C2447608901AA51217CA800D20440AD29F
:100BC300447608901AA81217CA78C5E6702575806E
:100BD300FE75902020950F304519C2457608901A6E
:100BE300AB1217CA800D20450AD2457608901AAE7B
:100BF3001217CA78C6E670257580FE759040209658
:100C03000F304619C2467608901AB11217CA800DE2
:100C130020460AD2467608901AB41217CA78C7E655
:100C230070257580FE75908020970F304719C24755
:100C33007608901AB71217CA800D20470AD2477652
:100C430008901ABA1217CA78C8E670257580FD7520
:100C5300900120900F304819C2487608901ABD12AF
:100C630017CA800D20480AD2487608901AC0121776
:100C7300CA78C9E670257580FD75900220910F3002
:100C83004919C2497608901AC31217CA800D204920
:100C93000AD2497608901AC61217CA78CAE670258E
:100CA3007580FD75900420920F304A19C24A760868
:100CB300901AC91217CA800D204A0AD24A760890A0
:100CC3001ACC1217CA78CBE670257580FD7590088B
:100CD30020930F304B19C24B7608901ACF1217CAC4
:100CE300800D204B0AD24B7608901AD21217CA787D
:100CF300CCE670257580FD75901020940F304C194B
:100D0300C24C7608901AD51217CA800D204C0AD20D
:100D13004C7608901AD81217CA78CDE670257580DC
:100D2300FD75902020950F304D19C24D7608901A0D
:100D3300DB1217CA800D204D0AD24D7608901ADEB9
:100D43001217CA78CEE670257580FD7590402096FF
:100D53000F304E19C24E7608901AE11217CA800D51
:100D6300204E0AD24E7608901AE41217CA78CFE6BC
:100D730070257580FD75908020970F304F19C24FF5
:100D83007608901AE71217CA800D204F0AD24F76C1
:100D930008901AEA1217CA78D0E670257580FB7599
:100DA300900120900F305019C2507608901AED121E
:100DB30017CA800D20500AD2507608901AF01217E5
:100DC300CA78D1E670257580FB75900220910F30AB
:100DD3005119C2517608901AF31217CA800D205187
:100DE3000AD2517608901AF61217CA78D2E67025FD
:100DF3007580FB75900420920F305219C252760809
:100E0300901AF91217CA800D20520AD2527608900E
:100E13001AFC1217CA78D3E670257580FB75900803
:100E230020930F305319C2537608901AFF1217CA32
:100E3300800D20530AD2537608901B021217CA78EA
:100E4300D4E670257580FB75901020940F305419EB
:100E5300C2547608901B051217CA800D20540AD27B
:100E6300547608901B081217CA78D5E6702575804A
:100E7300FB75902020950F305519C2557608901BAD
:100E83000B1217CA800D20550AD2557608901B0EF7
:100E93001217CA78D6E670257580FB7590402096A8
:100EA3000F305619C2567608901B111217CA800DBF
:100EB30020560AD2567608901B141217CA78D7E622
:100EC30070257580FB75908020970F305719C25796
:100ED3007608901B171217CA800D20570AD257762F
:100EE30008901B1A1217CA78D8E670257580F77513
:100EF300900120900F305819C2587608901B1D128C
:100F030017CA800D20580AD2587608901B20121752
:100F1300CA78D9E670257580F775900220910F3055
:100F23005919C2597608901B231217CA800D2059EC
:100F33000AD2597608901B261217CA78DAE670256A
:100F43007580F775900420920F305A19C25A7608AB
:100F5300901B291217CA800D205A0AD25A7608907C
:100F63001B2C1217CA78DBE670257580F77590087D
:100F730020930F305B19C25B7608901B2F1217CAA0
:100F8300800D205B0AD25B7608901B321217CA7859
:100F9300DCE670257580F775901020940F305C198E
:100FA300C25C7608901B351217CA800D205C0AD2EA
:100FB3005C7608901B381217CA78DDE670257580B9
:100FC300F775902020950F305D19C25D7608901B50
:100FD3003B1217CA800D205D0AD25D7608901B3E36
:100FE3001217CA78DEE670257580F7759040209653
:100FF3000F305E19C25E7608901B411217CA800D2E
:10100300205E0AD25E7608901B441217CA78DFE688
:1010130070257580F775908020970F305F19C25F38
:101023007608901B471217CA800D205F0AD25F769D
:1010330008901B4A1217CA78E0E670257580EF7591
:10104300900120900F306019C2607608901B4D12FA
:1010530017CA800D20600AD2607608901B501217C1
:10106300CA78E1E670257580EF75900220910F3004
:101073006119C2617608901B531217CA800D206153
:101083000AD2617608901B561217CA78E2E67025D9
:101093007580EF75900420920F306219C262760852
:1010A300901B591217CA800D20620AD262760890EB
:1010B3001B5C1217CA78E3E670257580EF759008FC
:1010C30020930F306319C2637608901B5F1217CA0F
:1010D300800D20630AD2637608901B621217CA78C8
:1010E300E4E670257580EF75901020940F30641935
:1010F300C2647608901B651217CA800D20640AD259
:10110300647608901B681217CA78E5E67025758027
:10111300EF75902020950F306519C2657608901BF6
:101123006B1217CA800D20650AD2657608901B6E74
:101133001217CA78E6E670257580EF759040209601
:101143000F306619C2667608901B711217CA800D9C
:1011530020660AD2667608901B741217CA78E7E6EF
:1011630070257580EF75908020970F306719C267DF
:101173007608901B771217CA800D20670AD267760C
:1011830008901B7A1217CA78E8E670257580DF7518
:10119300900120900F306819C2687608901B7D1269
:1011A30017CA800D20680AD2687608901B80121730
:1011B300CA78E9E670257580DF75900220910F30BB
:1011C3006919C2697608901B831217CA800D2069BA
:1011D3000AD2697608901B861217CA78EAE6702548
:1011E3007580DF75900420920F306A19C26A760801
:1011F300901B891217CA800D206A0AD26A7608905A
:101203001B8C1217CA78EBE670257580DF75900882
:1012130020930F306B19C26B7608901B8F1217CA7D
:10122300800D206B0AD26B7608901B921217CA7836
:10123300ECE670257580DF75901020940F306C19E3
:10124300C26C7608901B951217CA800D206C0AD2C7
:101253006C7608901B981217CA78EDE67025758096
:10126300DF75902020950F306D19C26D7608901BA5
:101273009B1217CA800D206D0AD26D7608901B9EB3
:101283001217CA78EEE670257580DF7590402096B8
:101293000F306E19C26E7608901BA11217CA800D0B
:1012A300206E0AD26E7608901BA41217CA78EFE656
:1012B30070257580DF75908020970F306F19C26F8E
:1012C3007608901BA71217CA800D206F0AD26F767B
:1012D30008901BAA1217CA78F0E670257580BF75AF
:1012E300900120900F307019C2707608901BAD12D8
:1012F30017CA800D20700AD2707608901BB012179F
:10130300CA78F1E670257580BF75900220910F3081
:101313007119C2717608901BB31217CA800D207120
:101323000AD2717608901BB61217CA78F2E67025B6
:101333007580BF75900420920F307219C2727608BF
:10134300901BB91217CA800D20720AD272760890C8
:101353001BBC1217CA78F3E670257580BF75900819
:1013630020930F307319C2737608901BBF1217CAEC
:10137300800D20730AD2737608901BC21217CA78A5
:10138300F4E670257580BF75901020940F307419A2
:10139300C2747608901BC51217CA800D20740AD236
:1013A300747608901BC81217CA78F5E67025758005
:1013B300BF75902020950F307519C2757608901B64
:1013C300CB1217CA800D20750AD2757608901BCEF2
:1013D3001217CA78F6E670257580BF75904020967F
:1013E3000F307619C2767608901BD11217CA800D7A
:1013F30020760AD2767608901BD41217CA78F7E6BD
:1014030070257580BF75908020970F307719C2774C
:101413007608901BD71217CA800D20770AD27776E9
:1014230008901BDA1217CA78F8E6702575807F7565
:10143300900120900F307819C2787608901BDD1246
:1014430017CA800D20780AD2787608901BE012170D
:10145300CA78F9E6702575807F75900220910F3068
:101463007919C2797608901BE31217CA800D207987
:101473000AD2797608901BE61217CA78FAE6702525
:1014830075807F75900420920F307A19C27A76089E
:10149300901BE91217CA800D207A0AD27A76089037
:1014A3001BEC1217CA78FBE6702575807F759008D0
:1014B30020930F307B19C27B7608901BEF1217CA5B
:1014C300800D207B0AD27B7608901BF21217CA7814
:1014D300FCE6702575807F75901020940F307C1981
:1014E300C27C7608901BF51217CA800D207C0AD2A5
:1014F3007C7608901BF81217CA78FDE67025758074
:101503007F75902020950F307D19C27D7608901B42
:10151300FB1217CA800D207D0AD27D7608901BFE30
:101523001217CA78FEE6702575807F759040209665
:101533000F307E19C27E7608901C011217CA800DE7
:10154300207E0AD27E7608901C041217CA78FFE622
:10155300702575807F75908020970F307F19C27F2B
:101563007608901C071217CA800D207F0AD27F7657
:1015730008901C0A1217CA75A0007590007840E6FF
:1015830070247580FED2B720B70F30F019C2F07601
:10159300089018DD1217CA800D20F00AD2F07608E1
:1015A3009018E01217CA7841E670247580FDD2B70F
:1015B30020B70F30F119C2F176089018E31217CA59
:1015C300800D20F10AD2F176089018E61217CA7836
:1015D30042E670247580FBD2B720B70F30F219C2F0
:1015E300F276089018E91217CA800D20F20AD2F297
:1015F30076089018EC1217CA7843E670247580F7C2
:10160300D2B720B70F30F319C2F376089018EF1250
:1016130017CA800D20F30AD2F376089018F2121736
:10162300CA7844E670247580EFD2B720B70F30F440
:1016330019C2F476089018F51217CA800D20F40A1F
:10164300D2F476089018F81217CA7845E670247514
:1016530080DFD2B720B70F30F519C2F5760890189E
:10166300FB1217CA800D20F50AD2F576089018FEF2
:101673001217CA7846E670247580BFD2B720B70F19
:1016830030F619C2F676089019011217CA800D2098
:10169300F60AD2F676089019041217CA7847E6704C
:1016A3002475807FD2B720B70F30F719C2F77608B9
:1016B3009019071217CA800D20F70AD2F7760890FF
:1016C300190A1217CAD2B220B2257532071217FDB2
:1016D3001217EF754801754900755000755100D513
:1016E30032037532011217F6D2B220B20280F0D261
:1016F300B320B3257532071218351217EF7548005A
:10170300754901755000755100D5320375320112C8
:1017130017F6D2B320B30280F0D2B420B4257532C9
:101723000712186D1217EF754800754900755001BF
:10173300755100D532037532011217F6D2B420B4B5
:101743000280F0D2B520B5257532071218A51217FD
:10175300EF754800754900755000755101D5320386
:101763007532011217F6D2B520B50280F0E5486054
:1017730005C2B2021794E5496005C2B3021794E5A6
:10178300506005C2B4021794E5516005C2B5021753
:101793009402007002003332C0D0C0E0C000D533E1
:1017A30004C2B0D2B67880E660011608B800F878B3
:1017B30040E660011608B848F8758CFAD000D0E00E
:1017C300D0D03232323232753310D2B0C2B6E49353
:1017D3003099FDC299F599A3E4933099FDC299F527
:1017E30099A3E4933099FDC299F599227E20DFFEF7
:1017F300DEFC227E60DFFEDEFC22753320D2B0C227
:10180300B63099FDC2997599C03099FDC299759901
:10181300003099FDC2997599C13099FDC2997599A6
:10182300003099FDC2997599C23099FDC299759995
:101833000022753320D2B0C2B63099FDC299759992
:10184300C03099FDC2997599013099FDC299759976
:10185300C13099FDC2997599013099FDC299759965
:10186300C23099FDC29975990122753320D2B0C255
:10187300B63099FDC2997599C03099FDC299759991
:10188300023099FDC2997599C13099FDC299759934
:10189300023099FDC2997599C23099FDC299759923
:1018A3000222753320D2B0C2B63099FDC299759920
:1018B300C03099FDC2997599033099FDC299759904
:1018C300C13099FDC2997599033099FDC2997599F3
:1018D300C23099FDC299759903229238408238002B
:1018E300923940823900923A40823A00923B4082D8
:1018F3003B00923C40823C00923D40823D00923E40
:1019030040823E00923F40823F009024408024006A
:101913009025408025009026408026009027408017
:101923002700902840802800902940802900902A91
:1019330040802A00902B40802B00902C40802C006C
:10194300902D40802D00902E40802E00902F4080BF
:101953002F00903040803000903140803100903231
:101963004080320090334080330090344080340014
:101973009035408035009036408036009037408067
:101983003700903840803800903940803900903AD1
:1019930040803A00903B40803B00903C40803C00BC
:1019A300903D40803D00903E40803E00903F40800F
:1019B3003F00904040804000904140804100904271
:1019C3004080420090434080430090444080440064
:1019D30090454080450090464080460090474080B7
:1019E3004700904840804800904940804900904A11
:1019F30040804A00904B40804B00904C40804C000C
:101A0300904D40804D00904E40804E00904F40805E
:101A13004F009050408050009051408051009052B0
:101A230040805200905340805300905440805400B3
:101A33009055408055009056408056009057408006
:101A43005700905840805800905940805900912485
:101A53004081240091254081250091264081260064
:101A630091274081270091284081280091294081B6
:101A73002900912A40812A00912B40812B00912C2F
:101A830040812C00912D40812D00912E40812E000C
:101A9300912F40812F00913040813000913140815E
:101AA30031009132408132009133408133009134CF
:101AB30040813400913540813500913640813600B4
:101AC3009137408137009138408138009139408106
:101AD3003900913A40813A00913B40813B00913C6F
:101AE30040813C00913D40813D00913E40813E005C
:101AF300913F40813F0091404081400091414081AE
:101B0300410091424081420091434081430091440E
:101B13004081440091454081450091464081460003
:101B23009147408147009148408148009149408155
:101B33004900914A40814A00914B40814B00914CAE
:101B430040814C00914D40814D00914E40814E00AB
:101B5300914F40814F0091504081500091514081FD
:101B6300510091524081520091534081530091544E
:101B73004081540091554081550091564081560053
:101B830091574081570091584081580091594081A5
:101B930059009224408224009225408225009226F7
:101BA3004082260092274082270092284082280004
:101BB300922940822900922A40822A00922B408255
:101BC3002B00922C40822C00922D40822D00922ECD
:101BD30040822E00922F40822F00923040823000AC
:101BE30092314082310092324082320092334082FD
:101BF300330092344082340092354082350092366D
:101C030040823600923740823700204D757A796BD7
:101C1300616E7420332076312E30692032303037B4
:101C23002D30322D3233202863294164616D2053D6
:101C33006D69616C656B206A616E6B6F6D757A7926
:101C43006B616E744077702E706C207777772E738C
:101C53006D69616C656B2E7072762E706C20577394
:101C63007A656C6B6965207072617761207A617344
:101C730074727A657A6F6E652E204A616B69656B43
:101C83006F6C7769656B207A6173746F736F7761BB
:101C93006E6961206B6F6D657263796A6E65206B27
:101CA3006F6475206E6965646F7A776F6C6F6E65AC
:101CB3002E20416C6C2052696768747320526573DF
:101CC30065727665642E204672656520666F7220A4
:101CD3006E6F6E20636F6D6D65726369616C206FEB
:051CE3006E6C792E205B
:00000001FF
